:020000040000FA
:06080000A2EF04F012005B
:02082A000000CC
:04082C002A0EF66E2C
:10083000080EF76E000EF86E00010900F550656FA6
:100840000900F550666F03E1656701D03DD00900EE
:10085000F550606F0900F550616F0900F550626F47
:1008600009000900F550E96E0900F550EA6E09002B
:1008700009000900F550636F0900F550646F090025
:100880000900F6CF67F0F7CF68F0F8CF69F060C0E5
:10089000F6FF61C0F7FF62C0F8FF0001635302E199
:1008A000645307E00900F550EE6E6307F8E2640751
:1008B000F9D767C0F6FF68C0F7FF69C0F8FF00010D
:0A08C0006507000E665BBFD712004B
:0608CA00FF0EE350036E77
:1008D000EF0E01D0F30EE76EE72E6CEF04F00C0E76
:1008E000026EE76AE72E72EF04F0022E71EF04F059
:0808F000032E6AEF04F0120070
:0808F8000F0EC1128B908B92D0
:10090000949094928B808B82FA0EE66E65EC04F0E4
:10091000E5528B908B92640EE66E65EC04F0E55226
:04092000F1D71200F9
:0C092400000EF36E00EE00F0080E01D88B
:100930001200EA6002D0EE6AFCD7F350E9601200C0
:04094000EE6AFCD788
:0C09440013EE00F023EE00F0F86A019CB6
:0C09500016EC04F07CEC04F0FDD7120063
:00000001FF
